:100000000C94AC070C94F0070C94F0070C94F007D8
:100010000C94F0070C94F0070C94F0070C94F00784
:100020000C94F0070C94F0070C94E6120C94B8139F
:100030000C94F0070C94F0070C94F0070C94F00764
:100040000C94F0070C94902C0C94F0070C94F0078F
:100050000C94F0070C9488220C94F0070C94F00791
:100060000C94F0070C94F0070C94F0070C94F00734
:100070000C94F0070C94F0070C94F0070C94F00724
:100080000C94F0070C94F0070C94F0070C94F00714
:100090000C94F0070C94F0070C94F0070C94F00704
:1000A0000C94F0070C94F0070C94F00725144714F7
:1000B0003515471435158C14AF143515041517155F
:1000C0005E185E188D188D18D1180F19291B291B61
:1000D0002819291B291A291AFD1A291B291B141B47
:1000E0000000F0A1F0A329002B000354E1003581AA
:1000F00000001E00140004001D7164004D001F006C
:100100001A0016001B00E1042A0020000800070066
:10011000060050002C0021001500090019004F00B6
:100120004A00220017000A00050000000254E00007
:10013000E3000000E20000002E77E400E70000008A
:10014000E60000002E7F23001C000B0011000000C1
:100150000454240018000D00100052004B0025002C
:100160000C000E00360051002C00260012000F007B
:100170003700E108280027001300330038713000F1
:100180004E002D002F003482E50031810000010077
:10019000010001000100010000003A0035003100BB
:1001A0000100010001003B00350221026400010052
:1001B0004C003C001E0224062202010001003D000A
:1001C0002D0224022404010001003E00010037003A
:1001D0001104000001000100010000000100000006
:1001E00001000100010000000100000001003F00CB
:1001F00024062402230200000100400022042502FC
:1002000035000100010041002304260235023700B9
:1002100001004200240425041F021E0201004300C5
:1002200031002604310201000100440045000100B4
:100230002D02010000000100010001000100010089
:1002400000000100010001000100010001000100A7
:100250000100F2000100010001000100F000F100C6
:100260000100F400010001000100F3000100F500AD
:100270000100010001000100010000000100010077
:100280000100000001000000010001000100000069
:100290000100000001000100010001000100000058
:1002A0000100010001000100A800A90001000100F7
:1002B00001000100AC00AA00B6000100010001002D
:1002C000AB0050000100010001000100520051008C
:1002D0000100AE000100010001004F00000001001C
:1002E0000100010001000100000001000100010007
:1002F00001000100010001000100010001000100F6
:1003000001000100010001000100010001000100E5
:1003100001000100010001000100010001000100D5
:1003200001000000010001000100000001000000C8
:1003300001000100010000000100000001000100B7
:1003400001000100010000000100010001000100A6
:100350000100010001000100010001000100010095
:100360000100010001000100010050000100010036
:1003700001000100520051000100010001000100D4
:1003800001004F0000000100010001000100010018
:100390000000010001000100010001000100010056
:1003A0000100500001000100010001005200510055
:1003B000010001000100010001004F0001000100E7
:1003C0000100010001000100010000000100010026
:1003D0000100000001000000010001000100000018
:1003E0000100000001003F00520051002302000004
:1003F00001004000240021001E00270001004100F0
:10040000250022001F0037000100420026002300C3
:1004100020002700010043003002300024022E009B
:1004200001004400450001000100010000000A0035
:100430002530313662003A200025303258000A72E9
:100440002F63203031323334353637383941424327
:100450004445460A000A002530325800626F756E26
:100460006365213A20006C656674207369646520B9
:1004700061747461636865640A006C6566742073F6
:10048000696465206E6F7420726573706F6E646945
:100490006E670A00747279696E6720746F207265E6
:1004A000736574206D637032333031380A000A444A
:1004B000454255473A20656E61626C65642E0A00BC
:1004C0005B735D004B6579626F6172642073746168
:1004D00072742E0A005B575D005B535D005B525DDA
:1004E000005B445D005B435D0016034500720067DE
:1004F000006F0044006F007800200045005A0000A3
:100500000016034500720067006F0044006F00781A
:1005100000200045005A0000000403090409028D70
:1005200000050100A0FA090400000103010100090F
:100530002111010001223F000705810308000A097B
:100540000401000103010200092111010001224DF3
:10055000000705820308000A0904020001030000E5
:10056000000921110100012236000705830308005C
:100570000A0904030002030000000921110100011F
:100580002220000705840320000107050403200042
:100590000109040400010300000009211101000108
:1005A0002239000705850310000112011001000027
:1005B0000008EDFE07130100010200010501090614
:1005C000A101050719E029E7150025019508750126
:1005D000810205081901290595057501910295010A
:1005E00075039101050719002977150025019578F4
:1005F00075018102C00631FF0974A101097515005A
:1006000025FF9520750881020976150025FF9520A4
:1006100075089102C005010980A10185021601003B
:1006200026B7001A01002AB700751095018100C095
:10063000050C0901A1018503160100269C021A017F
:10064000002A9C02751095018100C005010902A1D4
:10065000010901A1000509190129051500250195C8
:1006600005750181029501750381010501093009B4
:10067000311581257F950275088106093815812578
:100680007F950175088106050C0A38021581257FC2
:10069000950175088106C0C005010906A10105077D
:1006A00019E029E7150025019508750181029501DA
:1006B0007508810105081901290595057501910243
:1006C0009501750391010507190029FF150025FF04
:1006D000950675088100C00A002530325820006B4D
:1006E0006579626F6172645F7265706F72743A20CF
:1006F000000A0025303258006B6579626F617264C0
:100700005F7365745F6C65643A200064656C5F6B51
:1007100065795F6269743A2063616E27742064654D
:100720006C3A20253032580A006164645F6B657949
:100730005F6269743A2063616E2774206164643A71
:1007400020253032580A00646F6E652E0A00626FF1
:100750006F676D61676963207363616E3A202E2E47
:100760002E2000290A002575002F002575005D2820
:10077000002564002000256400200025640020007E
:100780002564007C0025303258006D6F7573656BF1
:100790006579205B62746E7C782079207620685DB4
:1007A000287265702F61636C293A205B006D6B5F66
:1007B000776865656C5F74696D655F746F5F6D61A7
:1007C00078203D2025640A006D6B5F776865656C55
:1007D0005F6D61785F7370656564203D2025640AF4
:1007E000006D6B5F74696D655F746F5F6D6178201C
:1007F0003D2025640A006D6B5F6D61785F737065E5
:100800006564203D2025640A006D6B5F696E746528
:100810007276616C203D2025640A006D6B5F646513
:100820006C6179203D2025640A006D6B5F776865F7
:10083000656C5F74696D655F746F5F6D6178203D95
:100840002025640A006D6B5F776865656C5F6D617C
:10085000785F7370656564203D2025640A006D6BC8
:100860005F74696D655F746F5F6D6178203D2025F1
:10087000640A006D6B5F6D61785F737065656420FD
:100880003D2025640A006D6B5F696E746572766148
:100890006C203D2025640A006D6B5F64656C617996
:1008A000203D2025640A000A00257500363A20778D
:1008B0006865656C5F74696D655F746F5F6D6178A5
:1008C0003A20000A00257500353A20776865656C86
:1008D0005F6D61785F73706565643A20000A00257A
:1008E0007500343A2074696D655F746F5F6D61786F
:1008F0003A20000A00257500333A206D61785F7355
:10090000706565643A20000A00257500323A206956
:100910006E74657276616C286D73293A20000A0046
:10092000257500313A2064656C6179282A31306D73
:1009300073293A20000A092D2056616C75657320D1
:100940002D0A004D3E004D25643E20003F0073659A
:10095000742064656661756C740A00433E200077FC
:10096000686572652064656C74613A2063757273A2
:100970006F723D25642C20776865656C3D25640A9F
:1009800053656520687474703A2F2F656E2E7769F1
:100990006B6970656469612E6F72672F77696B6927
:1009A0002F4D6F7573655F6B6579730A000A092DAA
:1009B000204D6F7573656B6579202D0A4553432F64
:1009C000713A09717569740A313A0964656C617923
:1009D000282A31306D73290A323A09696E746572BA
:1009E00076616C286D73290A333A096D61785F73FB
:1009F000706565640A343A0974696D655F746F5F88
:100A00006D61780A353A09776865656C5F6D617864
:100A10005F73706565640A363A09776865656C5F6F
:100A200074696D655F746F5F6D61780A0A703A0969
:100A30007072696E742076616C7565730A643A0928
:100A40007365742064656661756C74730A75703AB9
:100A5000092B310A646F776E3A092D310A70677578
:100A6000703A092B31300A7067646F776E3A092D3E
:100A700031300A0A7370656564203D2064656C74CA
:100A800061202A206D61785F7370656564202A207B
:100A900028726570656174202F2074696D655F74BC
:100AA0006F5F6D6178290A003F004D3E2000433E94
:100AB00020004C25640A000A092D20436F6E736FD5
:100AC0006C65202D0A4553432F713A09717569747D
:100AD0000A6D3A096D6F7573656B65790A000A09CD
:100AE0002D204D61676963202D0A643A09646562AF
:100AF00075670A783A096465627567206D6174727A
:100B000069780A6B3A096465627567206B6579627A
:100B10006F6172640A6D3A096465627567206D6F72
:100B20007573650A763A0976657273696F6E0A7332
:100B30003A097374617475730A633A09636F6E736B
:100B40006F6C65206D6F64650A302D343A096C61F5
:100B5000796572302D34284631302D4634290A50BB
:100B60006175733A09626F6F746C6F616465720AC4
:100B7000653A09656570726F6D0A6E3A094E4B529F
:100B80004F0A7A3A09736C656570204C45442074AD
:100B90006573740A000A002575002E6E6B726F3A39
:100BA00020000A002575002E737761705F62616313
:100BB0006B736C6173685F6261636B7370616365B3
:100BC0003A20000A002575002E737761705F677206
:100BD0006176655F6573633A20000A002575002E13
:100BE0006E6F5F6775693A20000A002575002E73E5
:100BF0007761705F72616C745F726775693A20002B
:100C00000A002575002E737761705F6C616C745FEC
:100C10006C6775693A20000A002575002E636170C3
:100C2000736C6F636B5F746F5F636F6E74726F6C06
:100C30003A20000A002575002E737761705F636F9C
:100C40006E74726F6C5F636170736C6F636B3A206C
:100C5000000A0025303258006B65796D61705F6362
:100C60006F6E6669672E7261773A20000A002575FB
:100C7000002E6D6F7573653A20000A002575002EF1
:100C80006B6579626F6172643A20000A0025750015
:100C90002E6D61747269783A20000A002575002E65
:100CA000656E61626C653A20000A0025303258009A
:100CB00064656275675F636F6E6669672E726177E0
:100CC0003A20000A0025750064656661756C745FE2
:100CD0006C617965723A20003F004E4B524F3A20CA
:100CE0006F66660A004E4B524F3A206F6E0A0074D0
:100CF000696D65725F636F756E743A202530346C70
:100D0000580A006B6579626F6172645F6E6B726F17
:100D10003A2025580A006B6579626F6172645F69D9
:100D2000646C653A2025580A006B6579626F6172C0
:100D3000645F70726F746F636F6C3A2025580A009D
:100D4000686F73745F6B6579626F6172645F6C6505
:100D5000647328293A2025580A000A092D20537463
:100D600061747573202D0A004743433A20342E39AD
:100D70002E33204156522D4C4942433A20312E38D1
:100D80002E31204156525F415243483A20617672DB
:100D9000350A004F5054494F4E533A204C55464166
:100DA00020424F4F544D41474943204D4F555345E5
:100DB0004B45592045585452414B455920434F4EBD
:100DC000534F4C4520434F4D4D414E44204E4B52C6
:100DD0004F203531320A004255494C443A203337CE
:100DE00030653930322D6469727479202832333A93
:100DF00033343A3037204465632032322032303188
:100E000035290A005649443A203078464545442859
:100E10004572676F446F7820455A29205049443AFB
:100E200020307831333037284572676F446F78202F
:100E3000455A29205645523A203078303030310A10
:100E400000444553433A20742E6D2E6B2E206B6563
:100E500079626F617264206669726D776172652074
:100E6000666F72204572676F646F780A000A092DF9
:100E70002056657273696F6E202D0A000A6D6F75BA
:100E800073653A206F66660A000A6D6F7573653A7E
:100E9000206F6E0A000A6B6579626F6172643A2096
:100EA0006F66660A000A6B6579626F6172643A2048
:100EB0006F6E0A000A6D61747269783A206F666617
:100EC0000A000A6D61747269783A206F6E0A000A2E
:100ED00064656275673A206F6E0A000A6465627520
:100EE000673A206F66660A000A0A626F6F746C6F59
:100EF000616465722E2E2E2000433E2000656563DE
:100F00006F6E6669673A0A00536C656570204C45E0
:100F10004420746573740A000000000000000000A3
:100F2000000000010204060A0F17202C3A4A5D71E6
:100F3000879DB3C7DAE9F5FCFFFCF5E9DAC7B39D95
:100F400087715D4A3A2C20170F0A0604020100003F
:100F5000000000000000000011241FBECFEFDAE007
:100F6000DEBFCDBF04B603FE24C08091F90190918D
:100F7000FA01A091FB01B091FC018730904BA74092
:100F8000B04BB9F41092F9011092FA011092FB01E2
:100F90001092FC0114BE84B7877F84BF88E10FB62E
:100FA000F89480936000109260000FBEE0E0FFE3D1
:100FB000099511E0A0E0B1E0ECEBFCE502C0059082
:100FC0000D92AA33B107D9F711E0AAE3B1E001C04D
:100FD0001D92A93FB107E1F70E941E100C945C2EF0
:100FE0000C940000FF93EF93E0913A01F0913B01E4
:100FF000309709F00995EF91FF910895FC018591D3
:10100000803011F0EFDFFBCF0895FF27E0E230E200
:1010100047FF0CC0419597FF09C0EDE260957095C0
:1010200080959095611D711D811D911D27FF02C046
:10103000219530E350E2AA27660F771F881F991F7A
:10104000AA1FA41710F0A41B63955A95A9F7AA30FC
:1010500008F0A95FA05DAF93F39561157105810557
:10106000910541F7ED3211F4EF93F395F21718F46F
:101070003F93F395FBCF8F91B5DFFA95E1F7089594
:10108000E991F9918591803021F0853219F0AADF3C
:10109000F9CF089520E0E89455915532C1F35033CB
:1010A00011F4689455915A3348F4505390F3220F39
:1010B000022E220F220F200D250FF4CF0EF42195C2
:1010C00089919991533619F3533729F1533559F1D1
:1010D000BC0188279927E8945C3621F4899199917D
:1010E00068945591543639F446EF7EF077FF0DC081
:1010F0008FEF9FEF0AC055374AE039F0583540E18D
:1011000021F0523642E009F00895FF93EF937DDF1E
:10111000EF91FF91B7CFFF93EF93FC018191803066
:10112000B9F360DFFBCFFF93EF9368DFF1CFDF937D
:10113000CF93CDB7DEB72596A3DFCF91DF9108958A
:1011400061110BC0FC018281882321F085EE0E9491
:10115000FB1603C085EE0E94C31780E090E008955F
:1011600008956091BC017091BD018091BE01909184
:10117000BF010E948B2156985E9825982D9826983D
:101180002E9827982F98823061F018F4813031F032
:101190000895833049F0843051F00895259A2D9AAE
:1011A0000895269A2E9A0895279A2F9A0895259A97
:1011B0002D9A279A2F9A089581EB98E0892B11F0A8
:1011C0000C94B108089556985E9825982D98269805
:1011D0002E9827982F988FEF90E090938900809316
:1011E000880090938B0080938A0090938D00809369
:1011F0008C00569A5E9A259A2D9A269A2E9A279AAC
:101200002F9A2FE782E490E1215080409040E1F74F
:1012100000C0000056985E9825982D9826982E9824
:1012200027982F98089589EA8093800089E0809319
:10123000810024982C983F988AB18F748AB96E984F
:10124000479A8BB1806B8BB9769A0E94E30880EB4A
:1012500098E0892B11F00C94B008089580E28093F7
:10126000000180913C0181110EC00E947D0981E046
:1012700080933C012FEF83ED90E32150804090401C
:10128000E1F700C0000080E40E9483098093000120
:1012900081112EC00E94AD0980930001811128C0E8
:1012A0000E94AD0980930001811122C08FE30E944A
:1012B000AD098093000181111BC00E94A50980E443
:1012C0000E94830980930001811112C08CE00E946A
:1012D000AD098093000181110BC00E94AD0980937C
:1012E0000001811105C08FE30E94AD0980930001C8
:1012F0000E94A5098091000108951092B9008AE02A
:101300008093B800089594EA9093BC009091BC003B
:1013100097FFFCCF9091B900987F983021F09031E1
:1013200011F081E008958093BB0084E88093BC00B5
:101330008091BC0087FFFCCF8091B900887F883105
:1013400011F0803471F780E0089584E98093BC0047
:101350008091BC0084FDFCCF08958093BB0084E89D
:101360008093BC008091BC0087FFFCCF9091B900B6
:10137000987F81E0983209F480E0089584E88093B2
:10138000BC008091BC0087FFFCCF8091BB0008951A
:1013900080910001811115C080E40E94830980932F
:1013A000000181110CC082E10E94AD09809300010F
:1013B000811105C08FEF0E94AD09809300010E944A
:1013C000A50984B1807F84B985B1807F85B98AB150
:1013D000837F8AB98BB1837F8BB93E9846980895F5
:1013E0000E942E09809300010E94C80980B38C706E
:1013F00080BB81B3836F81BBAEE3B1E0ECE4F1E08D
:101400008EE08E0F11921D928E13FCCF83E199E036
:10141000892B11F00C94130908959F92AF92BF92FB
:10142000CF92DF92EF92FF920F931F93CF93DF93B0
:10143000809100018823E1F080913D018F5F8093CE
:101440003D01811115C084E994E00E94FE070E94CD
:101450002E0980930001882329F08AE794E00E94F6
:10146000FE0706C086E694E00E94FE070E94E3089D
:101470000EE311E0C0E0D0E0BB24B39482E0A82EDC
:10148000CC24C394D12C27E5E22E24E0F22EC730E1
:10149000D10500F580910001811164C080E40E94B3
:1014A000830980930001811112C082E10E94AD097D
:1014B0008093000181110BC0C6010C2E01C0880F62
:1014C0000A94EAF780950E94AD09809300010E947A
:1014D000A50948C0CA30A1F028F4C83059F0C93075
:1014E00061F005C0CC3089F070F0CD3089F0209AE1
:1014F000289810C0219A29980DC0229A2A980AC0CB
:10150000239A2B9807C0529A01C0539A5B9802C045
:101510003E9A469890EA9A95F1F79FB1799902C060
:1015200082E001C080E091709B25982B7C9902C0DD
:1015300084E001C080E0892B7D9902C038E001C0C1
:1015400030E0832B7E9902C020E101C020E0822B95
:101550009FB19095991F9927991F9295990F907E09
:10156000892B10C080910001811174C080E40E9419
:10157000830980930001882309F459C0912C0E94AB
:10158000A509892DF8019081981739F18083809100
:101590000101882301F18091D70180FF04C08CE50F
:1015A00094E00E94FE078091D70180FF0CC08091DB
:1015B00001011F928F93FF92EF920E9497080F9064
:1015C0000F900F900F908091D70180FF04C085E5A8
:1015D00094E00E94FE07A09201010E94C809219692
:1015E0000F5F1F4FCE30D10509F051CF809101011F
:1015F0008823B1F0815080930101882339F08FE96D
:101600009FE00197F1F700C000000AC0ACE4B1E030
:10161000EEE3F1E0CF01825F91919D938E13FCCFB9
:101620008CED98E0892BC1F00E94DC0815C083E1A5
:101630000E94AD09809300018111A0CF81E40E9436
:10164000830980930001811199CF0E94BE09982ED1
:10165000909495CF80E096CF81E0DF91CF911F915C
:101660000F91FF90EF90DF90CF90BF90AF909F9041
:101670000895E82FF0E0E45BFE4F80810895CF925B
:10168000DF92EF92FF920F931F93CF93DF938EE33E
:1016900094E00E94FE078CE4E82E81E0F82EC0E082
:1016A000D0E099E3C92E94E0D92E00E314E0DF9353
:1016B000CF93DF92CF920E94970886E394E00E9436
:1016C000FE07F70181917F0190E00E94F1219F9335
:1016D0008F931F930F930E9497088EE294E00E94CD
:1016E000FE0721968DB79EB708960FB6F8949EBF59
:1016F0000FBE8DBFCE30D105D1F6DF91CF911F91B6
:101700000F91FF90EF90DF90CF9008958B3B910564
:1017100078F4883A910540F5853A9105D0F4843003
:10172000910508F0B1C08130910509F4ADC06BC0DE
:10173000803E910508F467C0883E910508F4A4C076
:101740009C01205F31092031310508F05CC09065B3
:101750000895853A910509F459C0863A910509F032
:1017600058C082E890E40895883A910509F454C07D
:10177000893A910509F453C08A3A910509F452C097
:101780008B3A910509F451C08C3A910509F450C087
:101790008D3A910509F44FC0803B910509F44EC084
:1017A0008E3A910509F44DC08F3A910509F44CC069
:1017B000813B910509F44BC0823B910509F44AC075
:1017C000833B910509F449C0843B910509F448C065
:1017D000853B910509F447C0863B910509F446C055
:1017E000873B910509F445C0883B910509F444C045
:1017F000893B910509F443C08A3B910509F442C035
:1018000080E094E4089580E090E0089581E890E419
:10181000089583E890E4089582EE94E4089589EEB3
:1018200094E408958AEE94E4089585EB94E4089591
:1018300086EB94E4089587EB94E408958CEC94E4AB
:1018400008958DEC94E4089583E895E408958AE87A
:1018500095E4089582E995E4089584E995E408956E
:1018600081E296E4089583E296E4089584E296E4A2
:10187000089585E296E4089586E296E4089587E265
:1018800096E408958AE296E40895089596E0799F93
:10189000F001112494E5899FE00DF11D1124E60F5C
:1018A000F11DEE0FFF1FEA51FF4F859194910895AE
:1018B000880F991FFC01E05AF0408591949108959A
:1018C000880F991FFC01E052FF4F85919491089574
:1018D00026E0729FF001112444E5849FE00DF11D84
:1018E0001124E60FF11DEE0FFF1FEA51FF4F859106
:1018F00094919C013A9521154FE1340708F41EC1DB
:101900003F512115304120F49F700E94600C0895D2
:101910009C0130532115304118F49927906C08959B
:10192000811520E5920769F40E944B1B4FEF84E379
:101930009CE0415080409040E1F700C000000C94D2
:10194000AD22813020E5920751F48EEA94E00E94A6
:10195000FE078091D70181608093D70108959C0193
:1019600030552115304108F051C0292F33272F70F1
:10197000332721303105D9F4AC014370552702C01B
:10198000220F331F4A95E2F73C68AC0164E0440F34
:10199000551F6A95E1F744275370242B352B73E0CC
:1019A000880F991F7A95E1F7807699271DC022301C
:1019B000310529F4982F8827816F906A0895233084
:1019C0003105A9F4AC014370552721E030E002C095
:1019D000220F331F4A95E2F73C6843E0880F991FB6
:1019E0004A95E1F7807E9770822B932B08952430DF
:1019F0003105E1F4AC014370552721E030E002C02D
:101A0000220F331F4A95E2F73A68E7CF9C0130571F
:101A10002115304118F49F70906208959C01305850
:101A20002115304118F49F70906A0895803E910509
:101A3000E0F4803C910558F58133910509F46FC0BD
:101A400048F48932910509F463C08A32910509F49A
:101A50006DC072C089339105E9F082389105D1F0EB
:101A60008533910509F44DC067C0833E910581F12E
:101A700038F4803E9105B9F0823E9105D9F05CC002
:101A8000863E910561F1873E9105A1F155C00E9406
:101A9000580C08952091EA0120FD02C021FF4CC09E
:101AA00080EE90E049C08091EA0180FFF9CF89E3A0
:101AB00090E042C08091EA0182FF0EC08091EA016D
:101AC00084FF03C080E090E037C083EE90E034C034
:101AD0008091EA0182FFF2CF82EE90E02DC08091EA
:101AE000EA0183FF0BC08091EA0184FDEBCF87EE12
:101AF00090E022C08091EA0183FFF5CF86EE90E06E
:101B00001BC08091EA0185FF07C089E290E014C004
:101B10008091EA0185FFF9CF85E390E00DC08091C7
:101B2000EA0186FF07C08AE290E006C08091EA01E0
:101B300086FFF9CF81E390E00E94860B0895089517
:101B400080916D0108959FB7F89410925C019FBF3A
:101B50009091F001943009F057C09091E9009F7086
:101B60003091EC00232F217030FD20E8922B24E0EF
:101B70002093E9002091EB0020FF43C02091EE006C
:101B800027FF3FC020915A01222321F02091E80035
:101B900025FF37C010925A0126E03091E80035FD4C
:101BA00015C03091F001343061F53091EB0035FD16
:101BB00028C0215021F481E080935A0122C0EFE92E
:101BC000FFE03197F1F700C00000E7CF8093F1000C
:101BD0008091E80085FD0AC08091E80080FFFCCF7D
:101BE0008091E8008E778093E80006C08FB7F89464
:101BF00021E020935C018FBF9F709093E90080E00B
:101C000008959F709093E9008FEF0895CF93DF932D
:101C100000D01F92CDB7DEB79C018091F0018430D7
:101C200019F593E099833B832A839093E9008FEF22
:101C30009091E800815095FD06C095ED9A95F1F7D9
:101C400000008111F5CF8091E80085FF0DC040E0D4
:101C500050E063E070E0CE0101960E94D6108091C2
:101C6000E8008E778093E8000F900F900F90DF913F
:101C7000CF910895CF93DF9300D01F92CDB7DEB7F9
:101C80002091F001243021F522E029839B838A836F
:101C900083E08093E9008FEF9091E800815095FDFB
:101CA00006C095ED9A95F1F700008111F5CF80916E
:101CB000E80085FF0DC040E050E063E070E0CE0139
:101CC00001960E94D6108091E8008E778093E800FC
:101CD0000F900F900F90DF91CF9108952091F00118
:101CE0002430F1F422E02093E9002FEF3091E80056
:101CF000215035FD06C035ED3A95F1F70000211170
:101D0000F5CF2091E80025FF0BC040E050E065E0F2
:101D100070E00E94D6108091E8008E778093E800F2
:101D20000895CF93DF932091F001243009F048C04B
:101D3000EC0180910C018823E1F080910D01882352
:101D4000C1F085E08093E9008FEF9091E800815029
:101D500095FD06C095E19A95F1F700008111F5CF48
:101D60008091E80085FF2CC040E050E060E170E029
:101D700017C081E08093E9008FEF9091E8008150D7
:101D800095FD06C095ED9A95F1F700008111F5CF0C
:101D90008091E80085FF14C040E050E068E070E00A
:101DA000CE010E94D6108091E8008E778093E800E3
:101DB00080E1FE01ADE5B1E001900D928A95E1F779
:101DC000DF91CF91089585EE94E00E94FE07809107
:101DD000EF01811109C00E946B120E94C81280910C
:101DE000E20084608093E200089581EE94E00E9416
:101DF000FE071092EF0108958DED94E00C94FE071C
:101E000089ED94E00E94FE070C947D2C85ED94E012
:101E10000E94FE070E9447220E94832C0E946D159B
:101E20000C949F0D20915B012F5F822F62E30E9433
:101E3000F12D992319F020935B01089510925B0115
:101E400080915C01882371F18091F001843041F52B
:101E50008091E9008F702091EC00922F917020FD0D
:101E600090E8892B94E09093E9009091EB0090FF2B
:101E700014C09091EE0097FF10C09091E80095FF7C
:101E800003C01092F100F9CF9091E80090FF05C0D7
:101E90009091E8009E779093E8008F708093E9001E
:101EA00010925C01089542E061EC81E00E94E5112E
:101EB00042E061EC82E00E94E51142E061EC83E0E7
:101EC0000E94E51142E261EC84E00E94E51142E1EA
:101ED00061EC85E00C94E5118091F201833009F406
:101EE00055C030F4813071F0823009F48EC008950D
:101EF0008A3009F47AC08B3009F460C0893009F067
:101F00009CC020C08091F101813A09F096C0809177
:101F1000E800877F8093E8008091F5019091F601B9
:101F2000892B21F460E18DE591E003C060E080E061
:101F300090E070E00E9421118091E8008B778093FF
:101F4000E80008958091F101813209F076C0809116
:101F5000F5019091F601009719F0049709F06DC012
:101F60008091E800877F8093E8008091E80082FDFF
:101F700005C08091F0018111F8CF5FC08091F10020
:101F800080936D018091E8008B7753C08091F101BF
:101F9000813A09F052C08091F5019091F601892BA8
:101FA00009F04BC08091E800877F8093E800809122
:101FB000E80080FFFCCF80910C0136C08091F101D8
:101FC0008132D9F58091F5019091F601892BA9F51F
:101FD0008091E800877F8093E8000E941A12809128
:101FE000F30180930C010C944B1B8091F101813221
:101FF00021F58091E800877F8093E8000E941A1203
:102000008091F40180936E0108958091F101813AED
:10201000A1F48091E800877F8093E8008091E80038
:1020200080FFFCCF80916E018093F1008091E800E9
:102030008E778093E8000C941A12089584B7877FF6
:1020400084BF88E10FB6F89480936000109260001E
:102050000FBE90E080E80FB6F894809361009093F3
:1020600061000FBE0E94FA150E946B120E94C812F6
:102070008091E20084608093E20083EA9DE00E9408
:10208000862178940E944D150E94FC1582E091E013
:102090000E9468150E946B2C84EC94E00E94FE075D
:1020A0008091F001853089F480EC94E00E94FE0775
:1020B0000E940B228091EE01882391F30E9433222B
:1020C000882371F30E94C010EBCF0E942A16E8CF3C
:1020D000292F332723303105C9F064F4213031052D
:1020E00081F02230310509F043C08DE890E02DE108
:1020F00035E042C021323105F1F02232310541F1A3
:1021000037C082E190E02AEA35E036C09927813075
:10211000910541F08230910541F0892B49F5E9E1C3
:10212000F5E005C0E1E0F5E002C0E9EEF4E08491FD
:1021300090E09F0121C06530D8F4E62FF0E0EE0F6B
:10214000FF1FEB5DFE4F2081318189E090E014C0DC
:10215000653070F470E0FB01EE0FFF1FE55EFE4F8F
:1021600020813181FB01EA5EFE4F808190E004C056
:1021700080E090E020E030E0FA0131832083089590
:1021800080E189BD82E189BD09B400FEFDCF809167
:10219000D8008F7D8093D8008091E000826080938A
:1021A000E0008091E00081FDFCCF0895CF92DF92A6
:1021B000EF92FF920F931F93CF93DF93EC018B016C
:1021C0006A010E943912811133C0C114D10439F05F
:1021D000F60180819181081B190BC80FD91FE12CD2
:1021E000F12C0115110519F18091E80085FD16C04B
:1021F0008091E8008E778093E800C114D10449F003
:10220000F60180819181E80EF91EF182E08285E07D
:102210000FC00E943912882321F30AC0899180934C
:10222000F10001501109FFEFEF1AFF0ADACF80E049
:10223000DF91CF911F910F91FF90EF90DF90CF90A2
:1022400008952091F7013091F8012617370748F0DB
:102250006115710539F42091E8002E772093E8008C
:1022600001C0B90140E061157105A9F12091F001AB
:10227000222309F443C0253009F442C02091E8002C
:1022800023FD40C02091E80022FD32C02091E800EB
:1022900020FFE9CF4091F3002091F20030E0342B91
:1022A000FC01CF016115710559F02830310540F46A
:1022B00081918093F100615071092F5F3F4FF1CF01
:1022C00041E02830310509F040E02091E8002E7708
:1022D0002093E800C8CF4111C9CF0AC08091F00116
:1022E000882361F0853061F08091E80083FD0AC0A9
:1022F0008091E80082FFF2CF80E0089582E00895A7
:1023000083E0089581E008952091F7013091F8016C
:102310002617370748F06115710539F42091E80058
:102320002E772093E80001C0B901FC0120E061157F
:10233000710591F18091F001882309F440C0853046
:1023400009F43FC08091E80083FD3DC08091E80022
:1023500082FD2FC08091E80080FFE9CF2091F3003B
:102360008091F20090E0922B6115710559F0883050
:10237000910540F424912093F10031966150710948
:102380000196F2CF21E0089709F020E08091E80063
:102390008E778093E800CBCF2111CCCF0AC08091FB
:1023A000F001882361F0853061F08091E80083FDC1
:1023B0000AC08091E80082FFF2CF80E0089582E0B9
:1023C000089583E0089581E00895982F973058F597
:1023D0009093E900981739F07091EC002091ED008E
:1023E0005091F00003C0242F762F50E021FF19C038
:1023F0003091EB003E7F3093EB003091ED003D7F5C
:102400003093ED003091EB0031603093EB0070932E
:10241000EC002093ED005093F0002091EE0027FF98
:1024200007C09F5FD3CF8F708093E90081E008954C
:1024300080E008958091F10187FF11C08091E8004C
:1024400082FD05C08091F0018111F8CF11C080910B
:10245000E8008B770BC08091F001882349F08091D0
:10246000E80080FFF8CF8091E8008E778093E80045
:1024700008952091E4003091E50095E64091EC004C
:10248000842F817040FF22C08091E80080FD1CC035
:102490008091F001882391F0853091F08091EB00DC
:1024A00085FD10C04091E4005091E50042175307AC
:1024B00029F39A01915011F784E0089582E008957C
:1024C00083E0089581E0089580E008954091E80058
:1024D00042FFDECF08950E94D9120E94E112E0EE81
:1024E000F0E0808181608083E8EDF0E080818F778B
:1024F000808319BCA7EDB0E08C918E7F8C93808196
:102500008F7E80831092EF0108950F931F93CF93D6
:10251000DF930E94D9120E94E112C8EDD0E08881B9
:102520008F77888388818068888388818F7D88837E
:1025300019BC1092F0011092EC011092EE01109271
:10254000ED0100EE10E0F80180818B7F80838881AF
:102550008160888342E060E080E00E94E511E1EE66
:10256000F0E080818E7F8083E2EEF0E08081816008
:102570008083808188608083F80180818E7F808362
:10258000888180618883DF91CF911F910F91089599
:10259000E8EDF0E080818F7E8083E7EDF0E08081E0
:1025A0008160808384E082BF81E08093EF010C949E
:1025B0008512E8EDF0E080818E7F80831092E2004A
:1025C00008951092DA001092E10008951F920F9280
:1025D0000FB60F9211242F933F934F935F936F93F6
:1025E0007F938F939F93AF93BF93EF93FF938091CC
:1025F000E10082FF0BC08091E20082FF07C0809162
:10260000E1008B7F8093E1000E94120F8091DA003D
:1026100080FF1FC08091D80080FF1BC08091DA002E
:102620008E7F8093DA008091D90080FF0DC080E119
:1026300089BD82E189BD09B400FEFDCF81E08093B0
:10264000F0010E94E30E05C019BC1092F0010E9437
:10265000F50E8091E10080FF19C08091E20080FFBB
:1026600015C08091E2008E7F8093E2008091E200AD
:1026700080618093E2008091D80080628093D800CE
:1026800019BC85E08093F0010E94000F8091E10069
:1026900084FF30C08091E20084FF2CC080E189BDBE
:1026A00082E189BD09B400FEFDCF8091D8008F7D05
:1026B0008093D8008091E1008F7E8093E10080912B
:1026C000E2008F7E8093E2008091E200816080933F
:1026D000E2008091EC01882311F084E007C0809132
:1026E000E30087FD02C081E001C083E08093F00138
:1026F0000E94060F8091E10083FF29C08091E200D3
:1027000083FF25C08091E100877F8093E10082E014
:102710008093F0011092EC018091E1008E7F809314
:10272000E1008091E2008E7F8093E2008091E200E0
:1027300080618093E20042E060E080E00E94E51169
:102740008091F00088608093F0000E94FC0EFF9161
:10275000EF91BF91AF919F918F917F916F915F9119
:102760004F913F912F910F900FBE0F901F90189592
:102770001F920F920FB60F9211242F933F934F93F6
:102780005F936F937F938F939F93AF93BF93CF93F9
:10279000DF93EF93FF93C091E900CF708091EC003D
:1027A000D82FD17080FDD0E81092E9008091F00020
:1027B000877F8093F00078940E94FC131092E900C8
:1027C0008091F00088608093F000CD2BCF70C09393
:1027D000E900FF91EF91DF91CF91BF91AF919F9170
:1027E0008F917F916F915F914F913F912F910F90BA
:1027F0000FBE0F901F9018951F93CF93DF93CDB707
:10280000DEB7AA970FB6F894DEBF0FBECDBFE1EFDB
:10281000F1E088E08E0F9091F10091938E13FBCF41
:102820000E946C0F8091E80083FF1FC18091F1012D
:102830009091F201492F50E04A30510508F015C13E
:10284000FA01EA5AFF4F0C94112E803881F0823839
:1028500009F00BC18091F5018F708093E9008091A0
:10286000EB0085FB882780F91092E90006C0809173
:10287000ED019091EE01911182609091E800977FB7
:102880009093E8008093F1001092F100C8C0282FC7
:102890002D7F09F0EAC0882319F0823061F0E5C08D
:1028A0008091F301813009F0E0C0933009F080E0BD
:1028B0008093EE012BC08091F301811127C080919C
:1028C000F5018F7009F4D1C08093E9002091EB00ED
:1028D00020FF1CC0933021F48091EB00806214C073
:1028E0009091EB0090619093EB0021E030E0A90122
:1028F00002C0440F551F8A95E2F74093EA001092F8
:10290000EA008091EB0088608093EB001092E90070
:102910008091E800877F86C08111A7C01091F301E4
:102920001F778091E3008078812B8093E300809172
:10293000E800877F8093E8000E941A128091E800E7
:1029400080FFFCCF8091E30080688093E300111149
:1029500002C082E001C083E08093F00186C080580D
:10296000823008F082C08091F3019091F4018C3D97
:1029700053E0950779F583E08A838AE289834FB72C
:10298000F894DE01139620E03EE051E2E32FF0E000
:1029900050935700E49120FF03C0E295EF703F5F32
:1029A000EF708E2F90E0EA3010F0C79601C0C0960D
:1029B0008D939D932F5F243149F74FBF8091E8009D
:1029C000877F8093E8006AE270E0CE0101960E9462
:1029D000211114C0AE014F5F5F4F6091F5010E945D
:1029E0006810BC01892B09F440C09091E800977FE2
:1029F0009093E80089819A810E9484118091E80077
:102A00008B778093E80031C0803879F58091E800B9
:102A1000877F8093E8008091EC018093F1008091A2
:102A2000E8008E778093E8000E941A121EC0811180
:102A30001CC09091F3019230C0F48091E800877F30
:102A40008093E8009093EC010E941A128091EC01AF
:102A5000811106C08091E30087FD02C081E001C0C2
:102A600084E08093F0010E94530F8091E80083FF7F
:102A70000AC08091E800877F8093E8008091EB0096
:102A800080628093EB00AA960FB6F894DEBF0FBE6B
:102A9000CDBFDF91CF911F910895CF938091F00129
:102AA0008823A1F0C091E900CF709091EC00892FAC
:102AB000817090FD80E8C82B1092E9008091E800B9
:102AC00083FD0E94FC13CF70C093E900CF9108955D
:102AD00090937401809373010895E0917301F091D4
:102AE0007401309721F00190F081E02D099480E08D
:102AF0000895EF92FF920F931F93CF93DF93E0918E
:102B00007301F09174013097B1F18C010280F3816F
:102B1000E02D09958091D70182FF2DC080FF04C070
:102B20008FED96E00E94FE07E80110E189EDE82EA6
:102B300086E0F82E8091D70180FF0BC088811F921C
:102B40008F93FF92EF920E9497080F900F900F9033
:102B50000F90115021961111EDCF8091D70180FF78
:102B60000AC087ED96E0DF91CF911F910F91FF9002
:102B7000EF900C94FE07DF91CF911F910F91FF9082
:102B8000EF900895E0917301F0917401309721F076
:102B90000480F581E02D0994089520917101309110
:102BA00072018217930771F0909372018093710103
:102BB000E0917301F0917401309721F00680F78164
:102BC000E02D0994089520916F01309170018217D2
:102BD000930771F09093700180936F01E0917301FE
:102BE000F0917401309721F00084F185E02D099473
:102BF000089508950C94F9150E9449220E94F00945
:102C00000C940F23CF93C82F8091D70182FF1EC051
:102C100080FF04C088EF96E00E94FE078091D701F4
:102C200080FF0CC01F92CF9383EF96E09F938F930A
:102C30000E9497080F900F900F900F908091D701EE
:102C400080FF04C081EF96E00E94FE078C2FCF9199
:102C50000C949F0DCF92DF92EF92FF920F931F93F0
:102C6000CF93DF93CDB7DEB72B970FB6F894DEBFC7
:102C70000FBECDBF0E940D0A86E7C82E81E0D82E78
:102C800000E010E0E02E802F0E94390BF601419108
:102C90006F01F42EF826B1F40F5F1F4F0E301105AF
:102CA00089F78FEF89838A831B820E945222816079
:102CB000782F9D838C8349815A816B818D810E94FD
:102CC000CD1640C09091D70191FF04C08B870E9420
:102CD0003F0B8B8520E030E04F2D50E0922FBA0162
:102CE000022E02C0759567950A94E2F760FF24C032
:102CF0002E83EF8221E030E0690102C0CC0CDD1CA4
:102D00009A95E2F790E08C219D21892B09F420E02F
:102D100028870E9452228160782F9A8789874E8166
:102D20005F8168858A850E94CD16F801EA58FE4FBA
:102D30008081C826C08206C02F5F3F4F26303105F4
:102D400069F6AACF0E948026109175010E946D1528
:102D50001817A1F00E946D15809375012B960FB680
:102D6000F894DEBF0FBECDBFDF91CF911F910F91C1
:102D7000FF90EF90DF90CF900C9402162B960FB639
:102D8000F894DEBF0FBECDBFDF91CF911F910F91A1
:102D9000FF90EF90DF90CF900895CF93DF93CDB762
:102DA000DEB72B970FB6F894DEBF0FBECDBF4F83B3
:102DB000588769877A878B87DE01119686E0FD0147
:102DC00011928A95E9F785E0FE01379601900D9200
:102DD0008A95E1F749815A816B817C818D819E8141
:102DE0000E94E51D2B960FB6F894DEBF0FBECDBF37
:102DF000DF91CF910895CF93882309F4C2C0C82FE3
:102E0000823859F40E946D1581FDBBC089E30E9490
:102E100081200E94602189E30CC0833879F40E94EC
:102E20006D1580FDAEC083E50E9481200E94602167
:102E300083E50E94D420CF910C946021843859F40A
:102E40000E946D1582FD9DC087E40E9481200E9432
:102E5000602187E4EECF8CEF8C0F813A48F48C2F01
:102E60000E94132B81118DC08C2F0E948120E3CFF3
:102E700080E28C0F883048F4C77081E001C0880F71
:102E8000CA95EAF70E942921D6CF8BE58C0F8330B3
:102E900078F4C53A29F0C63A31F083E890E005C0ED
:102EA00081E890E002C082E890E0CF910C94CD15CB
:102EB00088E58C0F833108F064C0C83A39F1C93A0B
:102EC00041F1CA3A49F1CB3A51F1CC3A59F1CD3AF4
:102ED00061F1C03B69F1CE3A71F1CF3A79F1C13B72
:102EE00081F1C23B89F1C33B91F1C43B99F1C53BF0
:102EF000A1F1C63BA9F1C73BB1F1C83BB9F1C93B50
:102F0000C1F1CA3BC9F180E090E038C082EE90E0A8
:102F100035C089EE90E032C08AEE90E02FC085EB9C
:102F200090E02CC086EB90E029C087EB90E026C0B3
:102F30008CEC90E023C08DEC90E020C083E891E021
:102F40001DC08AE891E01AC082E991E017C084E9C7
:102F500091E014C081E292E011C083E292E00EC0E1
:102F600084E292E00BC085E292E008C086E292E043
:102F700005C087E292E002C08AE292E0CF910C9411
:102F8000E315CF910895882309F44BC0823859F492
:102F90000E946D1581FF45C089E30E9481200E9437
:102FA000602189E30CC0833871F40E946D1580FFA5
:102FB00038C083E50E9481200E94602183E50E9441
:102FC000D4200C946021843859F40E946D1582FF3E
:102FD00028C087E40E9481200E94602187E4EFCF0F
:102FE0009CEF980F913A58F390E2980F983050F474
:102FF000877091E001C0990F8A95EAF7892F0E94A6
:103000002F21DFCF9BE5980F933020F480E090E0F4
:103010000C94CD15885A833120F480E090E00C9414
:10302000E3150895882321F00E9429210C94602142
:103030000895882321F00E942F210C946021089587
:10304000BF92CF92DF92EF92FF920F931F93CF9395
:10305000DF9300D000D000D0CDB7DEB725E0FC0173
:10306000DE01119601900D922A95E1F7FC01408155
:1030700031810281258122952F7063817481672BB4
:1030800009F4E7C23F3F19F44F3F09F4E2C27C0163
:1030900049833A8389819A812E830E944020182F88
:1030A000B92E0E943F200E94061FEB2DE295EF7083
:1030B000F0E0E05AFF4F2E810C94112E8B2D807F73
:1030C0009B2D9F70F92E882319F0F29480EFF8223F
:1030D000002349F0FF2009F469C28F2D0E94392195
:1030E0000E94602163C2812F0E94C317FF2009F450
:1030F000B0C28F2D0E943F2126960FB6F894DEBFF6
:103100000FBECDBFDF91CF911F910F91FF90EF9038
:10311000DF90CF90BF900C9460213B2D307F8B2DA2
:103120008F70303211F08295807F112319F01130A9
:1031300021F12DC00023B9F0222309F4A1C12130CF
:1031400009F09EC126960FB6F894DEBF0FBECDBF24
:10315000DF91CF911F910F91FF90EF90DF90CF9073
:10316000BF900C944921222319F0213009F471C237
:103170008E830E944C218E8197C1002321F026303E
:1031800008F067C27DC1253008F063C28DC10023FD
:1031900021F0222309F474C109C2222309F484C155
:1031A0001AC22B2D26952695237030E02115310566
:1031B00021F021303105D1F04CC2002321F0812FC4
:1031C0009B2D937002C080E090E026960FB6F89495
:1031D000DEBF0FBECDBFDF91CF911F910F91FF904A
:1031E000EF90DF90CF90BF900C94CD15002321F08D
:1031F000812F9B2D937002C080E090E026960FB641
:10320000F894DEBF0FBECDBFDF91CF911F910F911C
:10321000FF90EF90DF90CF90BF900C94E315812F3B
:10322000002319F00E94062502C00E946E252696F2
:103230000FB6F894DEBF0FBECDBFDF91CF911F91C7
:103240000F91FF90EF90DF90CF90BF900C94F325FB
:103250008B2D837009F07BC00111FBC1812F8295FA
:1032600086958770880F880F912F9F70C92ED12C5B
:10327000E12CF12C082E04C0CC0CDD1CEE1CFF1C34
:103280000A94D2F714FF12C04FE050E060E070E003
:1032900004C0440F551F661F771F8A95D2F7CB01D4
:1032A000BA01609570958095909503C060E070E0DC
:1032B000CB012B2D269526952370422F50E04230CE
:1032C0005105D9F04330510569F16C297D298E29CA
:1032D0009F294130510551F126960FB6F894DEBF73
:1032E0000FBECDBFDF91CF911F910F91FF90EF9057
:1032F000DF90CF90BF900C942D1F6C297D298E29D3
:103300009F2926960FB6F894DEBF0FBECDBFDF9182
:10331000CF911F910F91FF90EF90DF90CF90BF90D2
:103320000C94491F0E942D1FC701B60126960FB6A7
:10333000F894DEBF0FBECDBFDF91CF911F910F91EB
:10334000FF90EF90DF90CF90BF900C94111F00235F
:1033500019F08B2D817001C08695882309F479C1FD
:10336000812F829586958770880F880F912F9F7087
:10337000C92ED12CE12CF12C082E04C0CC0CDD1C64
:10338000EE1CFF1C0A94D2F714FF12C04FE050E06D
:1033900060E070E004C0440F551F661F771F8A95D8
:1033A000D2F7CB01BA01609570958095909503C0D6
:1033B00060E070E0CB012B2D269526952370422FDF
:1033C00050E042305105D9F04330510569F16C2984
:1033D0007D298E299F294130510551F126960FB63E
:1033E000F894DEBF0FBECDBFDF91CF911F910F913B
:1033F000FF90EF90DF90CF90BF900C9407206C2946
:103400007D298E299F2926960FB6F894DEBF0FBE20
:10341000CDBFDF91CF911F910F91FF90EF90DF9083
:10342000CF90BF900C9423200E940720C701B601C3
:1034300026960FB6F894DEBF0FBECDBFDF91CF91B9
:103440001F910F91FF90EF90DF90CF90BF900C9461
:10345000EB1F103FD1F118F4103E50F4A2C0123F00
:1034600009F464C008F44DC0133F09F474C099C056
:103470001F708B2D8F710023A1F00E94841F812F5C
:1034800026960FB6F894DEBF0FBECDBFDF91CF9169
:103490001F910F91FF90EF90DF90CF90BF900C9411
:1034A00012180E94A51F812F26960FB6F894DEBF32
:1034B0000FBECDBFDF91CF911F910F91FF90EF9085
:1034C000DF90CF90BF900C9419180023B1F02530F5
:1034D00008F0BFC08B2D8F7126960FB6F894DEBF13
:1034E0000FBECDBFDF91CF911F910F91FF90EF9055
:1034F000DF90CF90BF900C94CA1F263008F0A9C06F
:10350000E9CF0023A9F08B2D8F7126960FB6F89482
:10351000DEBF0FBECDBFDF91CF911F910F91FF9006
:10352000EF90DF90CF90BF900C94841F002359F34D
:103530008B2D8F7126960FB6F894DEBF0FBECDBFD0
:10354000DF91CF911F910F91FF90EF90DF90CF907F
:10355000BF900C94A51F002399F08B2D8F71269698
:103560000FB6F894DEBF0FBECDBFDF91CF911F9194
:103570000F91FF90EF90DF90CF90BF900C946F1F52
:1035800026960FB6F894DEBF0FBECDBFDF91CF9168
:103590001F910F91FF90EF90DF90CF90BF900C9410
:1035A000651F0023A9F0222309F4ADCF812F2696B1
:1035B0000FB6F894DEBF0FBECDBFDF91CF911F9144
:1035C0000F91FF90EF90DF90CF90BF900C94FB167F
:1035D000222309F4ADCF812F26960FB6F894DEBFD3
:1035E0000FBECDBFDF91CF911F910F91FF90EF9054
:1035F000DF90CF90BF900C94C3174B2D4F70612F6D
:10360000C7010E94A00826960FB6F894DEBF0FBE31
:10361000CDBFDF91CF911F910F91FF90EF90DF9081
:10362000CF90BF900C94891E4B2D4F70612FC70116
:1036300026960FB6F894DEBF0FBECDBFDF91CF91B7
:103640001F910F91FF90EF90DF90CF90BF900C945F
:10365000450C26960FB6F894DEBF0FBECDBFDF91A6
:10366000CF911F910F91FF90EF90DF90CF90BF907F
:1036700008950E9446210E941B210E9460210E9401
:1036800026270E94F32580E090E00E94CD1580E07F
:1036900090E00C94E3150E9436210C94391B0E9493
:1036A0004020292F22952F7030E02C3031054CF42A
:1036B0002A3031056CF4225031092230310588F46A
:1036C00007C02C30310549F02F30310531F009C0E9
:1036D000803E48F0803F29F406C093FB882780F99C
:1036E000089580E0089581E00895CF93DF9300D09E
:1036F00000D01F92CDB7DEB70F900F900F900F90B4
:103700000F90DF91CF910895CF93DF9300D000D039
:1037100000D0CDB7DEB726960FB6F894DEBF0FBE49
:10372000CDBFDF91CF9108951F93CF93DF93C091C9
:10373000840116E080918501C81799F0D0E01C9FA4
:10374000F0011D9FF00D1124EA57FE4F4081518179
:1037500062817381848195810E94841B2196C77048
:10376000E9CFDF91CF911F9108954091B60150911B
:10377000B7016091B8017091B9018091BA0190913F
:10378000BB010C94841B8091BB0182958F7009F062
:1037900054C08091B801882309F44FC080918401FE
:1037A000A09185016091B6017091B7014091B90176
:1037B0005091BA01B6E08A1709F43FC090E0411574
:1037C0005105C1F17F3F11F46F3FA1F1B89FF001A6
:1037D000B99FF00D1124EA57FE4F218172132AC0C0
:1037E0002081621327C02281211124C023813481CA
:1037F0002417350710F421503109241B350B283CC0
:103800003105C0F42091BB012F7020612093BB01D2
:1038100026E0289FF001299FF00D1124E557FE4F67
:1038200080818F708061808386EB91E00E942018F8
:103830000C94941B01968770BECF0895CF92DF92AF
:10384000EF92FF920F931F93CF93DF93CDB7DEB725
:1038500062970FB6F894DEBF0FBECDBF8C0185E036
:10386000F801DE011D9601900D928A95E1F7D801CD
:103870004C9111965C91119712966C911297139638
:10388000CD90DC9014973091B6017091B701809182
:10389000B9019091BA01009709F46BC17F3F19F407
:1038A0003F3F09F466C1E090B801EE2009F4C0C0C2
:1038B0002091BB01C816D90628F0F601E81BF90BC8
:1038C000CF0104C0809590958C0D9D1DFF24F3942D
:1038D000883C910578F0F12C207F09F0C6C07C2D42
:1038E000D98AC88A89890E94751B86EB91E00E945B
:1038F0002018B1C0822F807F09F046C0751314C014
:10390000341312C0611110C02F7020612093BB01CD
:103910000E94B51B86EB91E00E9420188091BB01AC
:10392000D80115968C932EC0CD2819F15F3F11F464
:103930004F3FF9F0F62E61111CC080918401209157
:10394000850136E0821709F45AC090E0389FF001F3
:10395000399FF00D1124EA57FE4F7181571306C0AD
:103960007081471303C07281711103C00196877083
:10397000E9CFF62E662309F418C18091BB0181605E
:103980008093BB01F12C11C1751308C0341306C01C
:10399000611104C08091BB01D801C3C04D875E870F
:1039A0008D859E856A8B0E944F1B6A898823E1F171
:1039B0006623D1F12091BB01822F82958F7090E018
:1039C000029774F08091B6019091B70198878F8328
:1039D0001986DB86CA862C87CE0107960E9420189E
:1039E00086E0F801A6EBB1E001900D928A95E1F72F
:1039F0000E94C31B0E94B51BFF24F394D6C04D87C1
:103A00005E878D859E850E944020292F22952F70EC
:103A100030E0223031050CF0BCC09F7009F0B6C018
:103A2000805E883008F4C1C0C8010E942018E4CF2D
:103A3000C816D90608F453C0F601E81BF90BCF01EC
:103A4000883C910508F450C0F12C7C2DD98AC88A95
:103A500089890E94751BE6EBF1E086E0DF011D928B
:103A60008A95E9F70E94B51BA0C0751314C03413E2
:103A700012C0611110C08091BB01F8018583C8019B
:103A80000E94201886E0E6EBF1E0DF011D928A95A6
:103A9000E9F7FE2C8AC04D875E878D859E856A8BEF
:103AA0000E944F1B6A89882309F4BECF662309F45C
:103AB000BBCF2091BB01822F82958F7090E002973F
:103AC0000CF48ECF8091B6019091B7019A838983CF
:103AD0001B82DD82CC822E83CE0101967FCF809522
:103AE00090958C0D9D1DACCFF62E662309F49CCFCE
:103AF00075132EC034132CC02091BB0120FD1FC0B4
:103B0000822F82958F70D9F0D80115962C93159736
:103B10008F3049F08F5F982F9295907F822F8F7012
:103B2000892B15968C93C8010E94201886E0F80115
:103B3000A6EBB1E001900D928A95E1F793CF86E074
:103B4000F801A6EBB1E001900D928A95E1F72DC046
:103B50004D875E878D859E850E944F1B811140CFCA
:103B60008091BB0181608093BB01C8010E94201835
:103B70001CC0662309F458CF4D875E878D859E85CE
:103B80000E944F1B882309F44FCF2ACF811148CFC1
:103B90000CC0243031050CF047CF9F7009F440CFA2
:103BA000F8019581907F09F03BCF8F2D62960FB67B
:103BB000F894DEBF0FBECDBFDF91CF911F910F9163
:103BC000FF90EF90DF90CF9008951F93CF93DF93F6
:103BD000CDB7DEB72C970FB6F894DEBF0FBECDBFC2
:103BE0004F83588769877A878B879C87CE01079692
:103BF0000E941E1C882369F08F8198852A853B8549
:103C0000232BF1F19F3F09F063C08F3F09F060C0A3
:103C100037C086E0FE013796DE01119601900D92C5
:103C20008A95E1F76F817885EA85FB85309741F1C8
:103C30007F3F11F46F3F21F12091850130E0C901F0
:103C40000196877099274091840150E08417950769
:103C500009F447C069837A83FD83EC8396E0929FE1
:103C6000D001939FB00D1124AA57BE4FFE0131968B
:103C700001900D929A95E1F7809385010E94941B23
:103C800016E080918401909185018917C1F1189FF8
:103C9000C00111248A579E4F0E941E1C882379F16F
:103CA000E09184011E9FF0011124EA57FE4F4081EC
:103CB000518162817381848195810E94841B8091EE
:103CC000840190E001968770992780938401D9CF71
:103CD0004F81588569857A858B859C850E94841BD8
:103CE000CFCF0E944B1B1092850110928401E6EB0E
:103CF000F1E086E0DF011D928A95E9F7C1CF2C96AD
:103D00000FB6F894DEBF0FBECDBFDF91CF911F91EC
:103D10000895EF92FF920F931F93CF93DF938C013F
:103D2000892B09F46CC0F12CEE24E394E801219670
:103D3000F8018491843740F4843008F051C0813018
:103D400081F0823019F15BC0853709F444C0A8F1D5
:103D50009CE7980F903708F052C08F770E94C317E6
:103D600041C00E5F1F4FFE01C49180E28C0F88306E
:103D700048F4C7708E2D01C0880FCA95EAF70E94DB
:103D8000392114C08C2F0E94FB162DC00E5F1F4FCF
:103D9000FE01C49180E28C0F883058F4C7708E2DDC
:103DA00001C0880FCA95EAF70E943F210E94602156
:103DB0001AC08C2F0E94C31716C00E5F1F4FFE0142
:103DC000C491CC2381F08FE99FE00197F1F700C007
:103DD0000000C150F6CF0E5F1F4FFE01F49003C0EC
:103DE0000E94FB168E018F2D882309F49FCFEFE9E7
:103DF000FFE03197F1F700C000008150F5CFDF916F
:103E0000CF911F910F91FF90EF90089508956093C7
:103E1000C0017093C1018093C2019093C3010C94BF
:103E2000391B0F931F930091C0011091C101209184
:103E3000C2013091C301DC01CB01802B912BA22B5D
:103E4000B32B8093C0019093C101A093C201B093A2
:103E5000C3011F910F910C94391B0F931F93009175
:103E6000C0011091C1012091C2013091C301DC0158
:103E7000CB0180239123A223B3238093C00190938D
:103E8000C101A093C201B093C3011F910F910C9483
:103E9000391B0F931F930091C0011091C101209114
:103EA000C2013091C301DC01CB0180279127A227F9
:103EB000B3278093C0019093C101A093C201B09336
:103EC000C3011F910F910C94391B1092BC011092E9
:103ED000BD011092BE011092BF010C94391B41E04C
:103EE00050E060E070E004C0440F551F661F771F6C
:103EF0008A95D2F74093BC015093BD016093BE01F7
:103F00007093BF010C94391B41E050E060E070E019
:103F100004C0440F551F661F771F8A95D2F7809102
:103F2000BC019091BD01A091BE01B091BF01482B91
:103F3000592B6A2B7B2B4093BC015093BD0160939E
:103F4000BE017093BF010C94391B41E050E060E06A
:103F500070E004C0440F551F661F771F8A95D2F783
:103F600040955095609570958091BC019091BD01F0
:103F7000A091BE01B091BF01482359236A237B233E
:103F80004093BC015093BD016093BE017093BF018B
:103F90000C94391B41E050E060E070E004C0440F35
:103FA000551F661F771F8A95D2F78091BC019091AB
:103FB000BD01A091BE01B091BF01482759276A27D2
:103FC0007B274093BC015093BD016093BE01709369
:103FD000BF010C94391B0F931F930091BC011091EA
:103FE000BD012091BE013091BF01DC01CB01802BCE
:103FF000912BA22BB32B8093BC019093BD01A09376
:10400000BE01B093BF011F910F910C94391B0F9308
:104010001F930091BC011091BD012091BE01309110
:10402000BF01DC01CB0180239123A223B323809322
:10403000BC019093BD01A093BE01B093BF011F913D
:104040000F910C94391B0F931F930091BC01109199
:10405000BD012091BE013091BF01DC01CB01802761
:104060009127A227B3278093BC019093BD01A09311
:10407000BE01B093BF011F910F910C94391B08959D
:10408000CF92DF92EF92FF920F931F93CF93DF9324
:104090008C01C090C001D090C101E090C201F090AD
:1040A000C3014091BC015091BD016091BE0170916E
:1040B000BF01C42AD52AE62AF72ACFE1D0E0D701EA
:1040C000C6010C2E04C0B695A795979587950A94BE
:1040D000D2F780FF07C0B8018C2F0E94680C813096
:1040E000910531F4219758F7B80180E00E94680CDF
:1040F000DF91CF911F910F91FF90EF90DF90CF90C4
:10410000089590910C01992321F090910D01911146
:1041100009C020910E0130910F01F90132969FEFF5
:1041200040E030C0982F9695969596959F30A0F4D4
:10413000E0910E01F0910F01E90FF11D877021E070
:1041400030E0A90102C0440F551F8A95E2F7CA0169
:104150009181892B818308959091D70190FF23C08D
:104160001F928F9389E297E09F938F930E94970805
:104170000F900F900F900F9008959F3F39F04F5F71
:104180004E3041F051915813F8CF0DC05111F7CF77
:10419000942FF5CF9F3F39F0F901E90FF11D97FDFD
:1041A000FA9582830895089590910C01992321F046
:1041B00090910D01911109C020910E0130910F01D4
:1041C000F9013296205F3F4F30C0982F9695969513
:1041D00096959F30A8F4E0910E01F0910F01E90F40
:1041E000F11D877021E030E0A90102C0440F551F86
:1041F0008A95E2F7CA018095918189238183089588
:104200009091D70190FF16C01F928F938BE097E09B
:104210009F938F930E9497080F900F900F900F908D
:1042200008953196E217F30729F090819813F9CF9A
:104230001082F7CF089581E090E0E0910E01F091B7
:104240000F01E80FF91F1082019680319105A9F73F
:1042500008959091D601892B8093D6010895809579
:104260009091D60189238093D60108951092D601AA
:1042700008959091D501892B8093D501089580955B
:104280009091D50189238093D50108951092D5018D
:1042900008958093C40108951092C40108958091F7
:1042A0000E0190910F01FC0131969C01205F3F4F60
:1042B00080E0919191118F5FE217F307D1F7089594
:1042C000E0910E01F0910F018091D6018083E09181
:1042D0000E01F0910F0190818091D501892B80838F
:1042E0008091C401882361F0E0910E01F0910F01EB
:1042F0009081892B80830E944F2181111092C401EB
:1043000080910E0190910F010C94791590933B01CF
:1043100080933A010895CF92DF92EF92FF926C0161
:10432000EE24FF24C114D104E104F10421F0C701FB
:10433000B60120E101C020E0C72ED82EE92EFF24CF
:10434000C114D104E104F10419F0285FC701B601DA
:104350006B017C0154E0F694E794D794C7945A9586
:10436000D1F7C114D104E104F10419F02C5FC701A5
:10437000B6016B017C0142E0F694E794D794C794B0
:104380004A95D1F7C114D104E104F10419F02E5F6C
:10439000C701B601DC01CB01B695A7959795879526
:1043A000892B8A2B8B2B09F02F5F822FFF90EF90A8
:1043B000DF90CF9008958295982F9C7C392F369569
:1043C0003695282F237344E0249FC0011124932F96
:1043D000982B292F2A7A2695892F8575880F822B6D
:1043E00008951F93CF93DF931F92CDB7DEB79983C4
:1043F0000E94DB21182F9981892F0E94DB21212F18
:1044000030E0322F2227A901482BCA010F90DF91FB
:10441000CF911F9108958091F001843009F110929D
:10442000D80120E488E190E00FB6F894A895809335
:1044300060000FBE2093600083B7817F846083BFDC
:1044400083B7816083BF7894889583B78E7F83BF5D
:1044500088E10FB6F89480936000109260000FBE60
:10446000089508950895CF930E9431220E940D0A65
:104470000E943222C0E08C2F0E94390B811104C0AF
:10448000CF5FCE30C1F701C081E0CF9108950C9489
:104490004B1B82E084BD93E095BD9AEF97BD80935E
:1044A0006E0008952FB7F8948091D9019091DA01A8
:1044B000A091DB01B091DC012FBF0895CF92DF9274
:1044C000EF92FF920F931F932FB7F8944091D90169
:1044D0005091DA016091DB017091DC012FBF6A011C
:1044E0007B01EE24FF248C0120E030E0C016D106D1
:1044F000E206F30610F4415051099A01281B390BCA
:10450000C9011F910F91FF90EF90DF90CF90089518
:104510001F920F920FB60F9211248F939F93AF9318
:10452000BF938091D9019091DA01A091DB01B09104
:10453000DC010196A11DB11D8093D9019093DA0190
:10454000A093DB01B093DC01BF91AF919F918F915C
:104550000F900FBE0F901F9018950E946B12F89449
:104560002FEF87EA91E6215080409040E1F700C0AC
:10457000000087E090EBDC018093F9019093FA0151
:10458000A093FB01B093FC019CE088E10FB6F89486
:10459000A895809360000FBE90936000FFCFEF92CC
:1045A000FF920F931F93CF93DF93D82FC0E08C2FF0
:1045B0000E94390B00E010E0E82EF12CC701002E1C
:1045C00002C0959587950A94E2F780FD06C00F5FBB
:1045D0001F4F0630110591F709C0602F7C2F80E036
:1045E0000E94460CD813F3CF81E004C0CF5FCE30D9
:1045F000F1F680E0DF91CF911F910F91FF90EF9046
:104600000895CF93C82F8CE20E94CF22882321F0F7
:104610008C2FCF910C94CF2280E0CF910895CF932F
:104620000E945E24811102C00E9444248EE497E01F
:104630000E94FE07C5E6C15049F00E940D0A8FE3B3
:104640009CE90197F1F700C00000F5CF87E497E0FF
:104650000E94FE0789E20E940123811113C18AE2B0
:104660000E94012381110E94442485E00E940123BD
:1046700081110E94AD220E9469248093D70187E0B6
:104680000E9401238823A9F18BE10E940123882342
:1046900051F08091D70181FB222720F991E09227E8
:1046A00090FB81F90EC08EE00E940123882361F007
:1046B0008091D70182FB222720F991E0922790FB7D
:1046C00082F98093D70115C080E10E940123909167
:1046D000D701882341F093FB222720F981E082272C
:1046E00080FB93F904C0892F809580FB90F990930B
:1046F000D7018091D7010E946D240E947B24809372
:10470000EA0180EE0E940123882341F08091EA01B2
:10471000982F909590FB80F98093EA0189E30E949D
:104720000123882359F08091EA0181FB222720F997
:1047300091E0922790FB81F98093EA0182EE0E943A
:104740000123882359F08091EA0182FB222720F976
:1047500091E0922790FB82F98093EA0186EE0E9415
:104760000123882359F08091EA0183FB222720F955
:1047700091E0922790FB83F98093EA0183EE0E94F7
:104780000123882359F08091EA0184FB222720F934
:1047900091E0922790FB84F98093EA0185E30E94DF
:1047A0000123882359F08091EA0185FB222720F913
:1047B00091E0922790FB85F98093EA0181E30E94C2
:1047C0000123882359F08091EA0186FB222720F9F2
:1047D00091E0922790FB86F98093EA0181E10E94A3
:1047E0000123882359F08091EA0187FB222720F9D1
:1047F00091E0922790FB87F98093EA018091EA018A
:104800000E947F248091EA0187FB882780F98093AA
:104810000D0187E20E940123C82F8EE10E9401232F
:104820008111C2608FE10E9401238111C46080E286
:104830000E9401238111C86081E20E94012381113D
:10484000C06182E20E9401238111C06283E20E9462
:1048500001238111C06484E20E940123882311F0A6
:10486000C06802C0CC2329F08C2F0E9476246C2FC4
:1048700003C00E947224682F70E080E090E0CF9126
:104880000C94071FCF9108956DEE7EEF80E090E0CD
:104890000E94472E60E082E090E00E94392E60E0A6
:1048A00083E090E00E94392E60E084E090E00E9476
:1048B000392E60E085E090E00C94392E80E090E0A5
:1048C0000E94332E21E08D3E9E4F09F020E0822F82
:1048D000089582E090E00C942B2E682F82E090E007
:1048E0000C94392E83E090E00C942B2E682F83E0FB
:1048F00090E00C94392E84E090E00C942B2E682FDD
:1049000084E090E00C94392E8091DF0180FF0BC091
:104910006091130185E0689FB0011124759567953A
:10492000759567952BC081FF09C06091130185E0E3
:10493000689FB00111247595679520C082FF07C05C
:104940006091130185E0689FB001112417C0909118
:10495000E0019923D1F060911201961788F7209118
:10496000130185E0289F90011124929FA001939F3D
:10497000500D112470E0CA010E94FD2D60387105B0
:1049800040F46115710539F002C065E070E0862FD2
:1049900008958FE7089581E008958091DF0180FFF9
:1049A00008C06091110170E07595679575956795E0
:1049B00021C081FF06C06091110170E07595679577
:1049C00019C082FF04C06091110170E010C0909185
:1049D000E0019923C1F0609110019617A0F7809132
:1049E0001101899FC001112470E00E94FD2D6038E3
:1049F000710528F46115710521F0862F08958FE760
:104A0000089581E0089561E070E0F4CF803F21F4E3
:104A10000E948424819504C0813F29F40E9484244B
:104A20008093E3010895823F21F40E9484248195BC
:104A300004C0833F29F40E9484248093E2010895F6
:104A4000893F19F40E94CD2405C08A3F31F40E94A9
:104A5000CD2481958093E40108958B3F21F40E9439
:104A6000CD24819504C08C3F29F40E94CD248093ED
:104A7000E5010895843F21F48091E101816017C030
:104A8000853F21F48091E101826011C0863F21F4CD
:104A90008091E10184600BC0873F21F48091E101A6
:104AA000886005C0883F31F48091E1018061809386
:104AB000E10108958D3F21F48091DF0181600BC0F9
:104AC0008E3F21F48091DF01826005C08F3F29F481
:104AD0008091DF0184608093DF010895803F39F485
:104AE0008091E30187FF6CC01092E30169C0813FB0
:104AF00029F48091E3011816BCF362C09091E201A1
:104B0000823F29F497FF5CC01092E20159C0833FB5
:104B100019F41916CCF354C0893F41F48091E40193
:104B200018160CF04DC01092E4014AC08A3F29F4D7
:104B30008091E40187FF44C0F6CF8B3F39F4809128
:104B4000E50187FF3DC01092E5013AC08C3F29F492
:104B50008091E5011816BCF333C0843F21F48091A5
:104B6000E1018E7F17C0853F21F48091E1018D7FA7
:104B700011C0863F21F48091E1018B7F0BC0873FFC
:104B800021F48091E101877F05C0883F31F4809155
:104B9000E1018F7E8093E10113C08D3F21F480916C
:104BA000DF018E7F0BC08E3F21F48091DF018D7F6E
:104BB00005C08F3F29F48091DF018B7F8093DF0157
:104BC0008091E20181110EC08091E30181110AC040
:104BD0008091E401811106C08091E501811102C03C
:104BE0001092E00108958091D70183FF7EC08AE88A
:104BF00097E00E94FE078091E1011F928F9385E864
:104C000097E09F938F930E94970883E897E00E9414
:104C1000FE078091E201282F332727FD30953F932F
:104C20008F9380E897E09F938F930E9497088EE779
:104C300097E00E94FE078091E301282F332727FD8C
:104C400030953F938F938BE797E09F938F930E94CC
:104C5000970889E797E00E94FE078091E401282FDA
:104C6000332727FD30953F938F9386E797E09F93F7
:104C70008F930E94970884E797E00E94FE07809137
:104C8000E501282F332727FD30953F938F9381E748
:104C900097E09F938F930E9497088EE697E00E947B
:104CA000FE078091E0011F928F938BE697E09F9320
:104CB0008F930E94970889E697E00E94FE078091F3
:104CC000DF011F928F9386E697E09F938F930E9458
:104CD000970883E697E00E94FE078DB79EB74C9633
:104CE0000FB6F8949EBF0FBE8DBF81EE91E00E947B
:104CF000C2150E9452229093DE018093DD01089537
:104D00001F93CF93DF938091DD019091DE010E948C
:104D10005E22AC019091E001992321F020911401D1
:104D200030E006C0209115018AE0289F90011124EF
:104D30004217530708F486C08091E201C091E30155
:104D4000D091E4011091E501811107C0C11176C035
:104D5000D11174C0111172C075C09F3F19F09F5FCF
:104D60009093E001181624F40E9484248093E201B9
:104D70008091E20187FF05C00E9484248195809381
:104D8000E2011C1624F40E9484248093E3018091A4
:104D9000E30187FF05C00E94842481958093E3018D
:104DA0006091E201662339F1C091E301CC2319F14E
:104DB000772767FD7095872F972F0E94022D23E399
:104DC00033E343E35FE30E94662D0E94CF2C6093A0
:104DD000E2016C2F772767FD7095872F972F0E9430
:104DE000022D23E333E343E35FE30E94662D0E9439
:104DF000CF2C6093E3011D1624F40E94CD248093F0
:104E0000E4018091E40187FF05C00E94CD248195D3
:104E10008093E401111624F40E94CD248093E501CF
:104E20008091E50187FF05C00E94CD248195809384
:104E3000E501DF91CF911F910C94F3259F3F09F07D
:104E40008ECF96CFDF91CF911F910895E1EEF1E0E3
:104E500085E0DF011D928A95E9F71092E00110923A
:104E6000DF0108958DEA99E00E94FE071F9281E01C
:104E70008F931F9285E08F938FE599E09F938F9397
:104E80000E9497080F900F900F900F900F900F9027
:104E900008958330E9F128F4813061F0823009F11E
:104EA0000895853009F462C008F449C0863009F4D9
:104EB00074C0089580911501262F30E0280F311D10
:104EC0002F3F310524F4680F6093150103C08FEF65
:104ED00080931501809115011F928F9388E998E0C6
:104EE00072C080911401262F30E0280F311D2F3F12
:104EF000310524F4680F6093140103C08FEF809391
:104F00001401809114011F928F9386E898E05BC092
:104F100080911301262F30E0280F311D2F3F3105DE
:104F200024F4680F6093130103C08FEF8093130183
:104F3000809113011F928F9383E798E044C0809182
:104F40001201262F30E0280F311D2F3F310524F4A8
:104F5000680F6093120103C08FEF8093120180915C
:104F600012011F928F938EE598E02DC08091110160
:104F7000262F30E0280F311D2F3F310524F4680F14
:104F80006093110103C08FEF809311018091110193
:104F90001F928F9385E498E016C080911001262F10
:104FA00030E0280F311D2F3F310524F4680F609346
:104FB000100103C08FEF80931001809110011F92A8
:104FC0008F938AE298E09F938F930E9497080F90A7
:104FD0000F900F900F900895833081F128F4813065
:104FE00059F08230D1F00895853009F449C0B8F104
:104FF000863009F456C0089580911501681720F491
:10500000861B8093150102C0109215018091150135
:105010001F928F938BE198E054C080911401681720
:1050200020F4861B8093140102C010921401809119
:1050300014011F928F9389E098E043C0809113017F
:10504000681720F4861B8093130102C0109213018D
:10505000809113011F928F9386EF97E032C0809169
:105060001201681720F4861B8093120102C010926F
:105070001201809112011F928F9381EE97E021C05F
:1050800080911101681720F4861B8093110102C0E2
:1050900010921101809111011F928F9388EC97E07B
:1050A00010C080911001681720F4861B80931001B6
:1050B00002C010921001809110011F928F938DEA0F
:1050C00097E09F938F930E9497080F900F900F90F7
:1050D0000F900895CF93C82F1F928F9382EB9AE081
:1050E0009F938F930E94970881E090E0A0E0B0E04A
:1050F000BC01CD0104C0660F771F881F991FCA9598
:10510000D2F70E94071F0F900F900F900F90CF9132
:105110000C944B1BCF938D3109F465C0B0F58E30E4
:1051200009F4CCC100F5873009F49BC1A8F486309E
:1051300009F06DC28091D701817F8E7F8093D70166
:1051400087EB9AE00E94FE0789EF9EE00E94FE072F
:1051500081E08093E70180C1883009F44FC08B3033
:1051600009F47CC154C2863109F4F0C138F48031AD
:1051700009F4B8C1813109F430C249C2893109F456
:10518000CEC18B3109F486C142C2853309F437C2DE
:1051900048F4873209F433C208F433C2893209F47F
:1051A0002EC235C2833438F48A3308F02CC28833D7
:1051B00009F454C12CC2833409F421C2883409F0A3
:1051C00026C20E944B1B88EE9EE00E94FE079FEFC6
:1051D00023ED80E3915020408040E1F700C00000C3
:1051E0000E94AD2239C188E09FE00E94FE070E9424
:1051F000892C0E946D150E949F0D2EC18DEF9EE09F
:105200000E94FE0788EC9CE00E94FE070E94722428
:105210001F928F9385EC9CE09F938F930E94970839
:1052200083EC9CE00E94FE070E946924C82F80EB5B
:105230009CE00E94FE071F92CF938BEA9CE09F9315
:105240008F930E94970889EA9CE00E94FE078FE9ED
:105250009CE00E94FE078C2F81701F928F938CE937
:105260009CE09F938F930E9497088AE99CE00E949C
:10527000FE0780E99CE00E94FE07C1FB882780F9B9
:105280001F928F938DE89CE09F938F930E949708C5
:105290008BE89CE00E94FE078FE79CE00E94FE07DF
:1052A000C2FB882780F91F928F938CE79CE09F9325
:1052B0008F930E9497088AE79CE00E94FE0781E78F
:1052C0009CE00E94FE07C3FBCC27C0F91F92CF933E
:1052D0008EE69CE09F938F930E9497088CE69CE05B
:1052E0000E94FE070E947B24C82F88E59CE00E9454
:1052F000FE071F92CF9383E59CE09F938F930E94BC
:10530000970881E59CE00E94FE0788E39CE00E94EC
:10531000FE078C2F81701F928F9385E39CE09F93F3
:105320008F930E9497088DB79EB780960FB6F8941A
:105330009EBF0FBE8DBF83E39CE00E94FE078CE101
:105340009CE00E94FE07C1FB882780F91F928F9383
:1053500089E19CE09F938F930E94970887E19CE0EE
:105360000E94FE0785E09CE00E94FE07C2FB8827A2
:1053700080F91F928F9382E09CE09F938F930E940D
:10538000970880E09CE00E94FE078EEE9BE00E9462
:10539000FE07C3FB882780F91F928F938BEE9BE05B
:1053A0009F938F930E94970889EE9BE00E94FE07CF
:1053B0008FED9BE00E94FE07C4FB882780F91F92B7
:1053C0008F938CED9BE09F938F930E9497088AEDBB
:1053D0009BE00E94FE0788EC9BE00E94FE07C5FB55
:1053E000882780F91F928F9385EC9BE09F938F9382
:1053F0000E94970883EC9BE00E94FE0787EA9BE0EF
:105400000E94FE07C6FB882780F91F928F9384EACB
:105410009BE09F938F930E94970882EA9BE00E94F3
:10542000FE078AE99BE00E94FE07C7FBCC27C0F974
:105430001F92CF9387E99BE09F938F930E949708D9
:1054400085E99BE00E94FE078DB79EB74C960FB68C
:10545000F8949EBF0FBE8DBFC1E0DEC08EED9AE016
:105460005BC08091D701C82FC17080FF09C08BED50
:105470009EE00E94FE078091D701817F8E7F47C00A
:105480008FEC9EE00E94FE078091D701816080939F
:10549000D701E2CF9091D70191FBCC27C0F981E0F1
:1054A000C827892FC0FB81F98093D701CC2319F03D
:1054B00082EC9EE027C084EB9EE02EC09091D70145
:1054C00092FBCC27C0F981E0C827892FC0FB82F965
:1054D0008093D701CC2319F085EA9EE013C085E9BB
:1054E0009EE01AC09091D70193FBCC27C0F981E0D0
:1054F000C827892FC0FB83F98093D701CC2351F0B3
:1055000089E89EE00E94FE078091D7018160809328
:10551000D70182C08CE79EE00E94FE079DCF8DE6FA
:105520009EE00E94FE0781E49EE00E94FE0784E068
:105530009EE00E94FE0787ED9DE00E94FE0783E942
:105540009DE00E94FE0788E69DE0E6CF8AE59DE0AB
:105550000E94FE070E946D151F928F9380E49DE0CC
:105560009F938F930E94970880910C011F928F93B5
:1055700089E29DE09F938F930E94970880916E012E
:105580001F928F9386E19DE09F938F930E949708CF
:1055900080910D011F928F9383E09DE09F938F93E5
:1055A0000E9497088091D9019091DA01A091DB01C6
:1055B000B091DC01BF93AF939F938F938FEE9CE0EC
:1055C0009F938F930E9497088DB79EB746960FB60C
:1055D000F8949EBF0FBE8DBF3FCF0E944B1BC09162
:1055E0000D0181E0C827C0930D01CC2329F085EE81
:1055F0009CE00E94FE0710C08AED9CE08DCF80E009
:1056000003C08D5101C089530E946A2825CF88EDBF
:105610009CE00E94FE07C0E08C2FCF91089580E0AF
:10562000089580E00895CF93C82F8091E7018130DD
:1056300081F020F0823009F44FC045C1E0910E01A5
:10564000F0910F018081813169F0823209F03DC112
:1056500009C0E0910E01F0910F018081813111F0BC
:10566000823261F48C2F0E940F2B811104C08C2F89
:105670000E948A282FC081E090E02CC08C2F0E94CD
:10568000112B811126C0C431E1F070F4CB3081F0D0
:10569000C031D1F40E9432278AEA9AE00E94FE07C4
:1056A00082E08093E70115C0C93259F0C83361F434
:1056B00087EB9AE00E94FE078EEA9AE00E94FE07BE
:1056C00008C01092E70103C188EA9AE00E94FE0731
:1056D000FEC081E08170FDC0C43220F5CE3108F0FB
:1056E000C0C0CB3099F1C8F4C73009F0D2C08AE00D
:1056F0008093150194E19093140193E0909313012A
:105700008093120188E08093110188E28093100158
:105710008EE499E00E94FE07BFC0C33149F1C43155
:10572000C1F0B7C0CB3409F4A9C028F4C93289F05C
:10573000C83361F0AEC0C13509F49EC0C23509F46A
:1057400099C0CE3409F0A5C06AE09EC00E943227FD
:10575000A3C08091E601882319F01092E6019CC055
:105760008BE599E00E94FE0781E08093E701B1C0DC
:1057700085E399E00E94FE0783E299E00E94FE071C
:10578000809115011F928F9380E299E09F938F93F0
:105790000E9497088EE199E00E94FE078CE099E054
:1057A0000E94FE07809114011F928F9389E099E077
:1057B0009F938F930E94970887E099E00E94FE07CD
:1057C00088EF98E00E94FE07809113011F928F934B
:1057D00085EF98E09F938F930E94970883EF98E05E
:1057E0000E94FE0782EE98E00E94FE07809112015F
:1057F0001F928F938FED98E09F938F930E9497084D
:105800008DED98E00E94FE0788EC98E00E94FE076C
:10581000809111011F928F9385EC98E09F938F9355
:105820000E94970883EC98E00E94FE078CEA98E0BB
:105830000E94FE07809110011F928F9389EA98E0E1
:105840009F938F930E94970887EA98E00E94FE0733
:105850008DB79EB748960FB6F8949EBF0FBE8DBF0A
:105860001BC0CE51EC2FF0E0E15DFE4F80818093B4
:10587000E60112C061E003C061E006C06AE0809109
:10588000E6010E94492708C08091E6010E94EC27AA
:1058900003C08CE499E013C08091E601882369F08D
:1058A0001F928F9386E499E09F938F930E949708AD
:1058B0000F900F900F900F9004C083E499E00E9426
:1058C000FE0781E006C01092E70180E002C080E0A0
:1058D00001CFCF910895E1E8F0E080818860808376
:1058E0008081816080838FB7F89493E090938900E2
:1058F00090ED909388008FBF0895EFE6F0E08081EF
:10590000826080830895EFE6F0E080818D7F808360
:105910000895EFE6F0E0908182E089278083089582
:105920001F920F920FB60F9211242F933F934F9314
:105930005F936F937F938F939F93AF93BF93EF93F7
:10594000FF938091E8019091E90101969093E9011C
:105950008093E801811103C082E00E949F0DE091D5
:10596000E901E695E695F0E0E85EF04FE49180917C
:10597000E8018E1303C080E00E949F0DFF91EF911C
:10598000BF91AF919F918F917F916F915F914F9157
:105990003F912F910F900FBE0F901F90189504D03C
:1059A0006894B1118DC0089570D088F09F5790F021
:1059B000B92F9927B751A0F0D1F0660F771F881F34
:1059C000991F1AF0BA95C9F712C0B13081F077D09B
:1059D000B1E0089574C0672F782F8827B85F39F039
:1059E000B93FCCF3869577956795B395D9F73EF493
:1059F00090958095709561957F4F8F4F9F4F08953B
:105A0000E89409C097FB3EF4909580957095619558
:105A10007F4F8F4F9F4F9923A9F0F92F96E9BB270E
:105A20009395F695879577956795B795F111F8CF8A
:105A3000FAF4BB0F11F460FF1BC06F5F7F4F8F4FF5
:105A40009F4F16C0882311F096E911C0772321F0EB
:105A50009EE8872F762F05C0662371F096E8862F83
:105A600070E060E02AF09A95660F771F881FDAF7DA
:105A7000880F9695879597F9089557FD9058440F8C
:105A8000551F59F05F3F71F04795880F97FB991F9D
:105A900061F09F3F79F0879508951216130614065A
:105AA000551FF2CF4695F1DF08C0161617061806E7
:105AB000991FF1CF86957105610508940895E894C2
:105AC000BB2766277727CB0197F908950BD078C0BD
:105AD00069D028F06ED018F0952309F05AC05FC045
:105AE0001124EECFCADFA0F3959FD1F3950F50E0BC
:105AF000551F629FF001729FBB27F00DB11D639F80
:105B0000AA27F00DB11DAA1F649F6627B00DA11D25
:105B1000661F829F2227B00DA11D621F739FB00DCB
:105B2000A11D621F839FA00D611D221F749F33273B
:105B3000A00D611D231F849F600D211D822F762FD4
:105B40006A2F11249F5750408AF0E1F088234AF0D1
:105B5000EE0FFF1FBB1F661F771F881F915050401D
:105B6000A9F79E3F510570F014C0AACF5F3FECF338
:105B7000983EDCF3869577956795B795F795E79509
:105B80009F5FC1F7FE2B880F911D9695879597F91A
:105B9000089597F99F6780E870E060E008959FEFAF
:105BA00080EC089500240A941616170618060906B4
:105BB000089500240A941216130614060506089583
:105BC000092E0394000C11F4882352F0BB0F40F40B
:105BD000BF2B11F460FF04C06F5F7F4F8F4F9F4F4B
:105BE0000895991B79E004C0991F961708F0961B39
:105BF000881F7A95C9F78095089597FB072E16F4AC
:105C0000009407D077FD09D00E94172E07FC05D01D
:105C10003EF4909581959F4F0895709561957F4FC3
:105C20000895EE0FFF1F0590F491E02D0994AA1B33
:105C3000BB1B51E107C0AA1FBB1FA617B70710F077
:105C4000A61BB70B881F991F5A95A9F780959095A9
:105C5000BC01CD010895F999FECF92BD81BDF89A9E
:105C6000992780B50895A8E1B0E042E050E00C9497
:105C70004E2E262FF999FECF1FBA92BD81BD20BDB1
:105C80000FB6F894FA9AF99A0FBE019608950E94F9
:105C9000392E272F0C943A2EDC01CB01FC01F99907
:105CA000FECF06C0F2BDE1BDF89A319600B40D9268
:0C5CB00041505040B8F70895F894FFCF21
:105CBC002002A00D910E6E0E3A0E060E0101C501CA
:105CCC0028080A03140A3F4D36203998064B06154E
:105CDC0006F505BC052F05480561057A059A0501F1
:0A5CEC000203040506070809000082
:00000001FF
